:020000020000FC
:1000000064CE00000000000020C0C2C194C0000007
:1000100000009EC000000000000000000203040673
:10002000080C10182030406080000406080C1018DE
:100030002030406080A0C00000070F1F3F000D0D62
:100040000403060D0503030202004FB662FD0EC055
:10005000552009F00994C52DC095089483FDC795D6
:10006000C4BDC093A10064604FBE1895C0916400E8
:10007000089483FDC795C4BDC093A1006B7FC09158
:100080006400CF3F09F420C070FF02C082FD05C0AC
:100090004FBEC19897989598189575FD0EC065FD4F
:1000A0000CC0C091B300C0FD9298C1FD9398C2FDF1
:1000B0009498CAEFC095CA95F1F7C198979895980A
:1000C0002092A1004FBE189524BCCC27C064C8BFA5
:1000D0006460F6CFC0CF70FFBECF65FDBCCFC19AC4
:1000E000BACF70FFB8CF65FDB6CF979AB4CF70FF87
:1000F000B2CF65FDB0CF959AAECF929A70FFABCFDD
:1001000065FDA9CFC7E0CA95F1F7C19AA4CF939A2C
:1001100070FFA1CF65FD9FCFC7E0CA95F1F7979A11
:100120009ACF949A70FF97CF65FD95CFC7E0CA9597
:10013000F1F7959A90CF4FB6C9B7CF7EC9BF6E7F02
:10014000CCB5CE0DDDB5DF1DDBBDCABD4FBE1895EC
:100150003FB68F7EA9B7A072A2118061A9B7AF7D0B
:10016000A9BFA9B7AE7FA9BF7894A0916800AA23C0
:1001700041F085FD2BC0A0916800AA95A09368006E
:1001800025C040E050E085FD15C0A6B396FDA095C2
:10019000A0FD4FEFAEB5A06496FDAF7BAEBDAA2724
:1001A000A062A8BF8D7FA6B396FDA095A0FD5FEFCE
:1001B000451739F7A0E461FDA093680085FD03C0F1
:1001C000A0E4A093680040939700816085FD0EC075
:1001D000A0916900AA2331F0A0916900AA95A0938B
:1001E000690004C08061AA27A062A8BF80FF0AC07E
:1001F000A09197004A2F61FF8E7F85FD01C000C04E
:10020000409361004091B600443009F004C0A091D1
:100210006100A0936300A52DA03408F06860A09150
:100220006000A395A093600059F0F894A9B7A1606D
:10023000A9BF84FF03C0A9B7A062A9BF3FBE18959C
:10024000A0917400A395A093740042E050916800BF
:10025000552329F085FF03C05A9550936800A0915B
:100260009700A13018F020929A000DC020929B00B8
:100270002092A500A0919A00AF5FA0939A0018F079
:10028000AFEFA0939A00B09061005091B600523049
:1002900049F466FF91F0A2E3BA1678F0A0918700C6
:1002A000A0936100533049F466FF39F0A2E3BA1617
:1002B00020F0A091C200A0936100509162005B15F4
:1002C00021F010F05A9501C05395509362004A9561
:1002D000D1F65091A500539509F45A955093A50075
:1002E000A091A600AA95A093A60009F046C0A1E09F
:1002F000A093A60045E0A091A7005A17F0F1A091A5
:10030000A8005A1728F441E0A3E0A093A60007C074
:10031000A091A9005A1718F441E04093A600D0908C
:100320009D00C0906300DC14A8F0A091B600A4303A
:10033000D9F066FD0FC0C0929D00539511F0A091B9
:10034000A700A093A500A1E0A093A600ACE3A09312
:10035000620013C0A0919D00A40F20F45FEF5093A2
:100360009D0002C0A0939D00A0919D00AF3F29F485
:10037000AFEFA0939B00A093A500F894A9B7A1604C
:10038000A9BF84FF03C0A9B7A062A9BF3FBE18954B
:100390003FB646B557B58F7EA9B7A072A21180614E
:1003A000A9B7AF7DA9BFA9B7AE7FA9BF789481FDDA
:1003B00025C0AEB5AF7B96FDA064AEBD8260A6B38E
:1003C00096FDA095A0FF05C0409365005093660080
:1003D0001FC1AEB5A06496FDAF7BAEBDAA27A062DB
:1003E000A8BF8D7F85FF01C006C140E0A6B396FD82
:1003F000A095A0FD00C140939700EFC0AEB5A064EA
:1004000096FDAF7BAEBD8D7F61FF72C0AEB5AF7B99
:1004100096FDA064AEBDAA27A062A8BF82604093EB
:10042000920050939300A09090004A19B0909100D0
:100430005B09BB24A22C4C38520518F4209296007C
:1004400049C0A091D600AA2359F1483C520528F48E
:10045000A0E1BA2EAAE0AA2E23C04836A1E05A078E
:1004600028F4A8E0BA2EAFE0AA2E1AC0403DA2E0C0
:100470005A0728F4A4E0BA2EAEE1AA2E11C0403AE1
:10048000A5E05A0728F4A2E0BA2EACE3AA2E08C0D1
:100490004839A8E05A0720F4A1E0BA2EA8E7AA2E0E
:1004A000C42EA0919400CA1AD52EA0919500DA0A04
:1004B000DD202AF4AFEFC094D094CA1ADA0A209251
:1004C0009600A8E0A210A0E0CA14DA0618F4A1E091
:1004D000A093960040939400509395004091920011
:1004E00050919300409390005093910002E075C0AA
:1004F000A09165004A1BA09166005A0B94FD60C054
:1005000093FD5EC092FD5AC086FF03C0D52EC42E57
:100510000CC05695479591FD51C05695479590FD55
:100520004DC0D52EC42ED694C79461FD19C0AC2DF4
:10053000AC51AD2DA24008F005C0DD2089F4AC2DF2
:10054000A85C70F4A0916700A395AA2311F0A09372
:100550006700AA3008F44FC02092970081604BC01A
:10056000A0916700AA2319F0AA95A0936700A22C76
:100570005091BC0097FD02C0A090CA00AAEFAA0E3D
:10058000A22DA21DCA18DA0A4FB74170442319F0F0
:1005900040E050E015C0AFEFCA16D20418F04FEF9C
:1005A00050E00EC0A091AE00CA9E412D000C441F29
:1005B00050E008F012C04FEF50E00FC0569547953D
:1005C00094FF07C0552309F04FEFA42FA6954A0FBB
:1005D000521D4F3F520508F04FEF40939700816046
:1005E00061FF09C0AFE1A095A923AB299A2F8F7DA8
:1005F000BB2009F48062A0E4A093680085FF03C0DB
:10060000AAE0A093680061FD03C085FD01C08F7E54
:1006100085FD03C0A0E2A0936900F894A9B7A1608A
:10062000A9BF84FF03C0A9B7A062A9BF3FBE1895A8
:1006300011E00AC013E008C01AE006C01EE104C0C1
:1006400014E602C018EC00C005E1BB27BA95F1F72B
:100650000A95D9F71A95C1F708952AE338E709C032
:1006600020E33CE806C02AE234EB03C025E238EC84
:1006700000C012E095FD9F7D95FF9062BB27939A85
:10068000BA95F1F7979ABA95F1F79798BA95F1F765
:100690009398BA95F1F7C19AB091AF00BA95F1F776
:1006A000C198B7E8BA95F1F71A9521F7022FB22F42
:1006B000BA95F1F70A95D9F73A95D9F6939A08952C
:1006C000221B39E0001F3A9509F40895221F211BCF
:1006D00018F4210F8894F6CF0894F4CF622C722C72
:1006E000B0E08894B395221F331FE0F73795279524
:1006F0008894912E802E020B130B10F4192D082DC7
:1007000010F4889401C00894661C771CBA9571F7A0
:10071000172D062D0895322D11232AF43A950095B0
:100720001095031B130BF894029F712C002D129F40
:10073000912C802C7894780C172D921C292DB4E0E4
:100740006B2E2695179507956A94D9F7332321F0D8
:1007500000951095031B130B08950091B60004300B
:1007600009F474C0B0919700B95198F0B72FB670E2
:1007700081F466FD2BC005E09090C800B92DBA95B4
:1007800021F00AE0BA9509F002E1B0917B00B01BBC
:10079000E0F066FF0AC0B0919F00B0939D00BFEFEC
:1007A000B093A500B1E0B093A600B0916100B09302
:1007B000630020927F00209280002092810020928E
:1007C0008200209283006F7B41C060649090C800DB
:1007D000B92DBA9579F4B0916200B095BB1FBB1FDB
:1007E0001B2FB7950B2FB12FB170B3951B2FB02FC7
:1007F000BE7F25C0B92DBA95BA9581F4B09162003B
:10080000B095BB1FBB1FBB1F1B2FB7950B2FB12F65
:10081000B370B3951B2FB02FBC7F14C0B091620092
:10082000B095BB1FBB1FBB1FBB1F1B2FB7950B2F4B
:10083000B12FB770B395B3951B2FB02FB87FB054BD
:100840000B2F120900937F001093800008951091E0
:100850007B00169500917A000795B0917F00B01B40
:100860000B2FB0918000B10B1B2F28F40038BFEF85
:100870001B0740F009C00F37120508F405C00FE749
:1008800010E002C000E81FEF009384001093850081
:10089000089500918400B09181000B0F10918500A4
:1008A000B09182001B1F20E03091850033230AF4B1
:1008B0002A95B09183002B1F1AF4203F40F00AC004
:1008C0002F3008F407C00FEF1FEF2FE003C000E048
:1008D00010E020EF30916300B0919C003B1718F4BA
:1008E000323030F009C0B0918500BB235AF004C00B
:1008F000B0918500BB2332F40093810010938200F5
:100900002093830008952091D80000918400000F67
:1009100010918500111FFFDE11232AF40038BFEF6C
:100920001B0740F009C00F37120508F405C00FE798
:1009300010E002C000E81FEF002352F0B091620007
:10094000B01B0B2F18F0013008F00AC001E008C0FE
:1009500000950F5FB09162000B0F08F001C00FEF20
:100960000093860008952091D90000918200109193
:100970008300D1DE11232AF40130BFEF1B0740F0C2
:1009800009C00F3F120508F405C00FEF10E002C0C8
:1009900001E01FEF112352F0B0918600B01B0B2F26
:1009A00018F0013008F00AC001E008C000950F5FA0
:1009B000B09186000B0F08F001C00FEF00936300A9
:1009C00008950FEF677F71FD29C072FD09C068604F
:1009D000B0917B00BA3020F0B52DB03408F4677FB9
:1009E000B091D500BB23D1F0B0917B00BB23B1F017
:1009F0000FEF10917B0064DEF894B091730072FDEC
:100A0000B5E00B9F112D002D7894112309F00FEF05
:100A1000B0919F000B1710F400919F0000939E006F
:100A2000089500917A0010917B0000541140B0911C
:100A30009E0010F4BA9501C0B39511F0B0939E00DA
:100A40000895EFD3B2E073FDB1E0B7B9B6B1B068C5
:100A5000B064B6B9EDDDB2E073FDB1E0B7B9B6B1DF
:100A6000B068B064B6B9B6B1B6FDFDCF04B115B18A
:100A7000B6B1BF77B6B926D42CE62093AA002223BC
:100A800009F441C030E03093AB00732E7694622EAF
:100A90006694620E731E262D372D0217130778F009
:100AA0008090AA00BCE6B80DB093AA008090AB007D
:100AB000B0E0B81DB093AB00260D371DEECF80908F
:100AC000AA009090AB001091AB0016950091AA007F
:100AD00007951695079523E0169507952A95E1F752
:100AE0002091B7002A9529F42092AA002092AB0009
:100AF0000AC02A9521F0800E911E2A95E1F7809276
:100B0000AA009092AB0008952091B700B6B1B6FD4F
:100B1000FBCF04B115B1B6B1BF77B6B9B091AC0097
:100B2000B395B093AC00B83060F12092AC00B091B6
:100B3000D400BB2321F1112329F0B091AD00BF3FB8
:100B400061F009C0B091AD000B1739F020F4BB2360
:100B500021F0BA9502C0B395E1F300919C00B093E7
:100B6000AD00BA3F50F400ECB93F38F400E8B83FAC
:100B700020F400E4B73F08F400E000939C00777F86
:100B800008952130B1F00F3FB3E01B0790F4BCE6AD
:100B9000BB2379F0B091AA000B17B091AB001B07F3
:100BA00040F4B0919C00BB2359F0BA95B0939C00DF
:100BB00007C0B0919C00BF3F19F0B395B0939C0063
:100BC00000919C00B0916300B01B10F40091630091
:100BD000B0919D000B1750F000919D00B0919D00C9
:100BE000BF3F21F0B0919D00B0939C00502E009328
:100BF0006400B091AC00B73009F47860089502E366
:100C0000F894B091DA000B9F012D000C001F78942E
:100C1000B0919C000B1710F000919C0000936100B4
:100C200000936300502E0093640000939F0008958A
:100C300020927A00B0EFB0937B000895F8940CB541
:100C40001DB5209174007894309175006090760005
:100C50000093750010937600031B160971FD03C005
:100C600076FD81C02BC07090770020937700270914
:100C7000222311F00FEF1FEF809078009090790001
:100C800030937800609279006918161910937C00EF
:100C900000917500109176000819190920917A00C9
:100CA00030917B0036952795020F131F10F40FEF3C
:100CB0001FEF00937A0010937B0029C020917A00E7
:100CC00030917B003901B4E08B2EB2E09B2E3430A2
:100CD00010F08A949A94383010F08A949A9476940A
:100CE00067948A94E1F726193709992021F016951F
:100CF00007959A94E1F7200F311F20937A003093E3
:100D00007B0028F43FEF30937A0030937B00323041
:100D100008F4706471FF02C0B3E00DC0B091C6006A
:100D200000917100023838F0B395003A08F0B3959D
:100D3000B63008F0B5E09B2EB4E08B2E10917B000E
:100D400000917A0024E0169507952A95E1F7081995
:100D5000120928F0B02FB250B12FB20910F402E0FE
:100D600010E0980126C020917A0030917B00390173
:100D7000769467946694669466942619320906956B
:100D80000695200F321D20937A0030937B0032307D
:100D900008F07F7B04E036952795369527952695B4
:100DA0002695201B10F0223008F422E08901909053
:100DB000C60060FDFECFE0908C00F0908D00616079
:100DC000B9B7B061B9BF380176FD44C07694679475
:100DD00000938C0010938D00B92DB330E1F0B0FD7D
:100DE00004C0060D171D930106C0000F111F02500D
:100DF000120922E030E0B92DB33068F020938E0064
:100E000030938F00009388001093890060928A00CD
:100E100070928B003DC000938E0010938F00209342
:100E200088003093890060928A0070928B0071FF75
:100E300010C0B0916D00B33060F000918F00109140
:100E40007C001595010F28F022F020928E0000936F
:100E50008F001EC0669400938C00B92DB33091F0C2
:100E6000B0FD03C0060D262D03C0000F025022E086
:100E7000B92DB33038F020938E0000938800609233
:100E80008A0006C000938E002093880060928A003A
:100E900000917D0002FD0350013029F495FD0AC048
:100EA000B0E0B7B909C0023019F4B7E0B7B904C06F
:100EB00095FDF6CFB6E0B7B90091A400000F10F48D
:100EC000BBE60B270093A40060FDFECFB2E0B09319
:100ED0006E006160B9B7B061B9BFB72FB670A1F04D
:100EE00020917A0030917B0036952795F8940CB5C7
:100EF0001DB5020F131F1BBD0ABD6160B0E1B8BF75
:100F0000B9B7B061B9BF78940895606120927E004E
:100F100020E067FD20E206C0606120927E0020E2B2
:100F200067FD20E0789401E076FD11C0B72FB67020
:100F300009F06F7EB0917B00B55048F002E0B550EB
:100F400020F003E0B55008F006E071FD0AE060FD16
:100F500012C0B0917E00BB2371F071FF08C0B09148
:100F60006D00B33020F0B0916E00BA9519F478940A
:100F700070615CC0AEDF789400000000F89476FDEC
:100F800016C010917B00173008F017E0B5E01B0F7A
:100F900072FD10E183FF110F62FF110F71FD12E866
:100FA000B4B56090A100B61990F2B10B80F2B0B761
:100FB000B77FB0BFB8B1B0B7B860B0BFB0917E0076
:100FC000B395B0937E00B8B176FD06C0B1E071FD77
:100FD000B2E0BA95F1F7B8B1B072B21709F01BC020
:100FE00071FF05C003950A3008F00395B0CF64FF88
:100FF00099CF6F7E3CB56DB470907A0080907B0085
:10100000370D681C6BBC3ABD6160B0E1B8BFB9B7C1
:10101000B061B9BF87CFB0916D00B23008F482CF14
:1010200064FD80CF0A9509F092CF7F7E20918E00DB
:1010300030918F00F894B0E1B8BF0CB51DB5020F28
:10104000131F1BBD0ABDE0908800F090890061600D
:10105000B9B7B061B9BF7894B72FB67039F0B09115
:101060006D0072FFB395B0936D0009C074FF07C0A7
:1010700067FD05C064FD03C0BF91BF91D9C4089549
:1010800000E063FF03C064FF01C001E0F894109129
:101090007100B7E01B9F212D102D7894200F26950D
:1010A0001795269517952695179510937100183763
:1010B00018F4B8E7B093710000917100B09172001C
:1010C0000B1720F06062C1989798959860FDFECF4D
:1010D000E0908A00F0908B006160B9B7B061B9BF51
:1010E0000895B2E095FD07C0F894B0937D00939AFF
:1010F00092987894E5C0F894B0937D00939A949870
:101100007894DEC0B3E082FF24C095FD11C002E0F8
:10111000F894B0937D00E7E8F0E00093B300959871
:10112000949A62FF02C0979A01C093987894C8C0BD
:1011300002E0F894B0937D00E7E8F0E00093B3009C
:10114000C198929A62FF02C0979A01C093987894CE
:10115000B7C095FD0BC0F894B0937D00E1E7F0E0D7
:10116000959862FF01C0979A7894AAC0F894B093BA
:101170007D00E1E7F0E0C19862FF01C0979A7894A2
:101180009FC0B4E095FD07C0F894B0937D00929A9B
:101190009498789495C0F894B0937D00949A92981E
:1011A00078948EC0B5E082FF24C095FD11C001E0A7
:1011B000F894B0937D00EDE7F0E00093B3009798CA
:1011C000939A62FF02C0C19A01C09298789478C045
:1011D00004E0F894B0937D00E1E9F0E00093B300FF
:1011E0009798939A62FF02C0959A01C09498789458
:1011F00067C095FD0BC0F894B0937D00EBE6F0E07E
:10120000979862FF01C0C19A78945AC0F894B0933D
:101210007D00E7E7F0E0979862FF01C0959A789427
:101220004FC0B6E095FD07C0F894B0937D00949A46
:101230009398789445C0F894B0937D00929A9398CF
:1012400078943EC0B1E082FF24C095FD11C004E057
:10125000F894B0937D00E1E9F0E00093B300C19809
:10126000929A62FF02C0959A01C09498789428C01F
:1012700001E0F894B0937D00EDE7F0E00093B30057
:101280009598949A62FF02C0C19A01C0929878948E
:1012900017C095FD0BC0F894B0937D00E7E7F0E030
:1012A000C19862FF01C0959A78940AC0F894B093EF
:1012B0007D00EBE6F0E0959862FF01C0C19A78945A
:1012C0006F7D08952AE630E0F9012092B300C198BD
:1012D00097989598929A939A949A6B7F0895A4EB15
:1012E000B0E007E00D9307E00D9301E00D9304E0FB
:1012F0000D930FEF0D930D9309E00D9302E00D9305
:1013000001E00D9301E00D93A0ECB0E001E00D933E
:1013100000E00D9304EB0D930FEF0D930D930D93E0
:1013200003E00D930FEF0D9301E00D930FEF0D937D
:1013300005E20D9300ED0D9308E70D9308EC0D9376
:1013400004E00D930FEF0D9301E00D9300E00D937A
:101350000AE70D930AE00D9300E00D9301E00D9371
:1013600000E00D930FEF0D9308952091BB008B7F4C
:10137000233009F48460B091BC009F7DB1FD906280
:101380009F7BB091BD00B1FD9064223011F0886068
:1013900001C0877F08950A95E00FF21DB49108956A
:1013A000ECE1F0E00091B400F6DFB093D800ECE19E
:1013B000F0E00091B500EFDFB093D900EAE2F0E091
:1013C0000091BA00E8DFB093DA000091D300002367
:1013D00009F40395013108F001E1B02FB00FB00F0F
:1013E000B093A7001B2FB10FB10FB00FB093A8009F
:1013F000B10FB00FB00FB093A900B091D0000FEFB4
:101400001CE0B23011F400EA1AE0B33011F402E843
:1014100015E00093720010937300E8E3F0E0009190
:10142000D700B9DFB093A200089508952091CA00B3
:101430003091CB00B091BC00B33009F43E5097FF1F
:1014400002C020E03FEFB32FB21B6B2EB25810F456
:10145000B2E86B2E00E00395609EB12DBD57D8F326
:101460000093AE0008959068E1DFE8D820E030E016
:10147000B0E16B2EDFD8B09197002B0F321D6A942C
:10148000C9F7B4E036952795BA95E1F7822E9F7794
:10149000CDDF0895F894E3E0F0E0B9E0B7BFB49190
:1014A000B078C1F3F894A895B1B5B861B1BDB0E01A
:1014B000B1BDB4E0BEBFBFE5BDBF04DFB0E0B8BBA7
:1014C000B2E1B7BBB0E0B5BBB0E0B4BBBCE1B2BB0E
:1014D000BCEBB1BB2224A0E0B0E02D92AA31E9F729
:1014E000A0E6B0E00FEF2D920A95E9F7B1E0B093D6
:1014F000A400F5DED2D2B6B1B460B6B90091CC008A
:101500000093AF00B1E0B0936A00F8949BD8A5D8DF
:1015100095D8A6D893D8A7D891D84ED393D892D897
:101520008FD8F8940AEF1AEFA6B396FDA095A0FF06
:101530001FC01A95C9F70A95B1F7E0E0FCE1B59133
:10154000B43E39F4B591B03E21F4B591BF3F09F4F2
:101550000CC0E0E0F395F395B591B83F49F4B5912F
:10156000B43931F4B591BA3A19F4EE27F6950994E5
:10157000FCDE16DF5ADF5ADF0091CC000093AF008B
:10158000A1DEB2E0B3BFB2E0BEBDB2E0B5BDB1E531
:10159000B8BFB9BFB0B7B77FB0BFB8B1B0B7B86068
:1015A000B0BF46D878944DDABEB5B06496FDBF7B27
:1015B000BEBDB9B7B062B9BFBB27B062B8BF8D7F3F
:1015C00041D8626033E02CE0B0919600BB2321F457
:1015D0002CE03A9509F4A5CF31D880FFA2CF8E7FB9
:1015E000B0919700B23078F3B92FBF710091990094
:1015F00000939800B0939900B01729F72A9521F726
:101600006D7FBEB5B06496FDBF7BBEBDBB27B0622B
:10161000B8BF8D7FB091D600BB2321F48062B92F73
:10162000B0709B2F8F7B209267000AD885FF05C082
:10163000B0916700BA3008F08064FCD702E085FF03
:1016400001C000E0B0919700B017B8F3F89405D846
:1016500004D803D87894F6D720928700EBD7B091BE
:10166000C000B13008F46EC0B0916A00B13008F427
:1016700069C085FD18C0B0919700BF3F08F462C0F3
:10168000F894F4D77894DCD7B0919700B130C0F7D4
:10169000F894E3D7D1D7E1D77894D2D7B091970017
:1016A000BF3FB0F3BBC2B8E09B2E9068F894BEDE9B
:1016B0007894C6D7F8949F77B9DE80909700B09160
:1016C0009700BF37789408F445C0B2D7F894CED7C6
:1016D00078949A9451F7C7DEB82DB550B093CB00EB
:1016E000B1D7F89407D26DD27894BAE09B2E906867
:1016F000F8949CDE7894A4D7F8949F7797DE809036
:101700009700B0919700BF37789478F791D7F89405
:10171000A4D792D7A2D778949A9449F7A4DEB82D8B
:10172000BB5FB093CA008ED7F894E4D159D27894B5
:1017300087D7F8947BDE7894B0919700BF3F08F488
:1017400098CF6CC200919700B09187000B1710F0F2
:101750000093870075D701E0B091BC00B35009F445
:1017600005E0B0919700B01708F078CFF8947ED7D5
:101770007DD77CD7789466D720926A0020926B0040
:1017800020926C00B0916B00B395B0936B00BF3F9B
:1017900069F5B0916C00B395B0936C00B091CE0038
:1017A00009E1BA9559F002E3BA9541F00DE7BA950F
:1017B00029F00AEFBA9511F020926C00B0916C00FC
:1017C000B017A0F0B0916C00BA95B0936C00B4EB78
:1017D000B0936B00B091CD00B093AF00F89446D7B2
:1017E0007894B091CC00B093AF002AD725D7B091B0
:1017F0006800BB2319F485FF01C093CE01E085FD8D
:1018000001C006E0B0919700B01708F4BBCF18D71D
:10181000B0916800BB2309F484CEF89453DD209284
:1018200061002092620020926300522C209264009A
:101830002092A3007894B091B900BB0FB093A000A0
:1018400020927F00209280002092810020928200CE
:10185000209283002092AC0060E070E02092710042
:10186000B8E0B093AC007860E3D6B2E073FDB1E0CD
:10187000B7B9B6B1B068B064B6B9B6B1B6FDFDCF10
:1018800004B115B1B6B1BF77B6B9112309F00FEFA6
:101890000093AD0039D9B8E0B093AC007860809087
:1018A000BB00B2E0B093BB0060DD8092BB00F89457
:1018B000BFEFB0939C00A3D9B0916100B0939C009E
:1018C000B0939D00B0939E007894B1E0B093610016
:1018D000B09363005B2EB0936400B093A600B09108
:1018E0009B00B093A500B091BC00B33019F49F7D6C
:1018F00087FD90627160726020926D0092DCA2DCC4
:1019000097D99CD995D99AD993D906C0F8942DDD49
:1019100078942092AC00777FFFDA1FD7B1DBE1DB50
:101920008DD9F3DA66FD93D776FF4BD876FD79D85B
:10193000A7DBE8DB83D9F0DA66FDABD7A1DB21DCDE
:101940007DD9E3DA66FDDFD79BDB2CDC77D9E4DADF
:1019500066FD09D895DB65DC71D9D7DAB2E073FD95
:10196000B1E0B7B9B6B1B068B064B6B989DB6ADCCA
:1019700065D9CAD871FF20C067FD1EC0B0919F0015
:10198000B0939C00B0939D00B0919B00B093A500D4
:10199000B1E0B093A60018E12CE0B0916D00B11752
:1019A00028F07D7F746020936F0006C0B09197008F
:1019B000B13008F0B1CF46C072FF10C067FD0EC055
:1019C000B0916F00BA9511F47B7FA0CFB0936F00F8
:1019D000B0919700B13008F09FCF34C020927000D2
:1019E000B0919A00B13058F0B0919F00B0939D0033
:1019F000B0919B00B093A500B1E0B093A600B09168
:101A00009A000AEFB01708F01DC085FF04C0B0911E
:101A10006800BB23B9F000EF67FF05C0B0919F00DD
:101A2000B0939C0000E2B0917B00B01708F474CF33
:101A3000B0917000B395B0937000B0919700BB2344
:101A400009F002C020927000F8943CDC8090BB004A
:101A5000B2E0B093BB0089DC8092BB0020926100B1
:101A60002092620020926300522C20926400209207
:101A7000A0007E7F7894DCD525DCB6B1B460B6B921
:101A800085FF05C0B0916800BB2309F44ACDB09131
:101A9000C100B13008F0D1CD71CEEDE0F0E023D03F
:101AA000053A09F01BC0EEE0F0E01DD00A3509F060
:101AB00015C03AE0A4EBB0E0E3E0F0E014D00D9301
:101AC00031963A95D9F738E1A0ECB0E0EFE0F0E0DC
:101AD0000AD00D9331963A95D9F702C000DC0AD0AE
:101AE000E7E2F0E00895E199FECFEEBBFFBBE09A9C
:101AF0000DB308951ED03AE0A4EBB0E0E3E0F0E0CF
:101B00000D910FD031963A95D9F738E1A0ECB0E0BD
:101B1000EFE0F0E00D9105D031963A95D9F712D06B
:101B20000895E199FECF0DBBEEBBFFBBE29AE19AAF
:101B30000895EDE0F0E00FEFF4DFEEE0F0E00FEFFE
:101B4000F0DF0895EDE0F0E005EAEBDFEEE0F0E035
:101B50000AE5E7DF08953091B0000091B10031301F
:101B600011F40093B400323011F40093B500333017
:101B700011F40093B600343011F40093C8003530EE
:101B800011F40093B700363011F40093BA003730E7
:101B900011F40093C600383011F40093BB003930C3
:101BA00011F40093D0003A3011F40093BC003B30A4
:101BB00011F40093BD00089525E044D52A95E9F776
:101BC00008954BD54DD54FD551D536D546D548D5A9
:101BD0004AD54CD531D541D543D545D547D50895BE
:101BE00045D541D53DD539D527D540D53CD538D576
:101BF00034D522D53BD537D533D52FD50895809010
:101C0000B0009090B10029D528D527D515D58A9454
:101C1000D1F72CD511D59A94E1F70895F894D1DF36
:101C20007894CADFC9DFB1E0B093B000B1E0B093FF
:101C3000B1002092B200F894E2DF7894B5E06B2E08
:101C400070909700FFD4B09197007B16C9F7B13020
:101C500018F0BF3F40F107C07EDFF8944BDFB1DFE3
:101C6000B8E0B1BDA9DF6A9459F7B091B200B3955D
:101C7000B093B200B33008F4DECF9EDFB091B10074
:101C8000B395B093B100F894B091B000BA95EEE37B
:101C9000F0E0EB0FF21D049178940395B091B10040
:101CA000B01708F4C6CF88DF87DFB091B000B395D6
:101CB000B093B000B091B000BC3008F4B7CF0FDBE8
:0C1CC000F89418DFB8E0B1BD77DFE4CB8A
:00000001FF
